:040000002500780B54
:0A00100029000000E902090AFF08B8
:10010000FF0FFF0FFF0FFF0FFF0FFF0FFF0FFF0F7F
:10011000FF0FFF0FFF0FFF0FFF0FFF0FFF0FFF0F6F
:10012000FF0FFF0FFF0FFF0FFF0FFF0FFF0FFF0F5F
:10013000FF0FFF0FFF0FFF0FFF0FFF0FFF0FFF0F4F
:10014000FF0FFF0FFF0FFF0FFF0FFF0FFF0FFF0F3F
:10015000FF0FFF0FFF0FFF0FFF0FFF0FFF0FFF0F2F
:10016000FF0FFF0FFF0FFF0FFF0FFF0FFF0FFF0F1F
:10017000FF0FFF0FFF0FFF0FFF0FFF0FFF0FFF0F0F
:10018000FF0FFF0FFF0FFF0FFF0FFF0FFF0FFF0FFF
:10019000FF0FFF0FFF0FFF0FFF0FFF0FFF0FFF0FEF
:1001A000FF0FFF0FFF0FFF0FFF0FFF0FFF0FFF0FDF
:1001B000FF0FFF0FFF0FFF0FFF0FFF0FFF0FFF0FCF
:1001C000FF0FFF0FFF0FFF0FFF0FFF0FFF0FFF0FBF
:1001D000FF0FFF0FFF0FFF0FFF0FFF0FFF0FFF0FAF
:1001E000FF0FFF0FFF0FFF0FFF0FFF0FFF0FFF0F9F
:1001F000FF0FFF0FFF0FFF0FFF0FFF0FFF0FFF0F8F
:100200000A0C040B6600800A28002A002A03CA018F
:100210002A03CA012A03CA012A03CA012A03CA01FE
:100220002A03CA012A03EA01050C0809020C0A067E
:10023000010C26000E0C08090000FF0C2600080C1B
:1002400008096600080C08092600070C0807290B96
:10025000170C000008096600080C08092600070CA6
:100260002807330B170C000008096600080C080962
:100270002600070C48073D0B170C00000809660014
:10028000080C08092600070C6807470B170C00002C
:1002900008096600080C08092600070C8807510B9E
:1002A000170C000008096600080C08092600070C56
:1002B000A8075B0B170C000008096600080C08096A
:1002C0002600070CC807650B170C0000080966001C
:1002D000080C08092600FC0C0600060C08090000A2
:1002E000020CE807010C740B26000E0C0809020B27
:0E02F000C70C0200FF0C2600FC0C0600020BDF
:021FFE00FA0FD8
:00000001FF
